:020000040000FA
:02000000A22834
:08000800F000030EF1000408F2
:10001000F2000A08F3008A01831203138B1A0B1DE6
:1000200014287E200B1175280B1A8B1C1A28962079
:100030008B1075288B190B1C202897200B10752806
:100040000B1F752883160C1F2B2883120C1F2B28BF
:1000500098200C13752883168C1E332883128C1E4F
:1000600033289920752883160C1E3C2883120C1EF9
:100070003C289A200C12752883168C1D4528831263
:100080008C1D45289B208C11752883160C1D4E282D
:1000900083120C1D4E289C200C11752883168C1C75
:1000A000572883128C1C57289D208C107528831686
:1000B0000C1C602883120C1C60289E200C107528D4
:1000C00083160D1E692883120D1E69289F200D12AC
:1000D000752883168D1D722883128D1D7228A0200D
:1000E0008D1175288312A1200D1073088A007208E3
:1000F0008400710E8300F00E700E0900A00B080042
:10010000043085062330A00081309F00E530A10037
:10011000A10B88281F15000000001F198B281E083E
:1001200086002030A100A10B9328080008000800D9
:10013000080008000800080008000800080008007F
:1001400008000800831203138501860187018316C6
:100150000E309F003B308500003086000030870065
:100160008730810020308B0000308C0000308D0003
:100170008312203084008001840A841FBB2823302E
:0C018000A0008C018D018B17C528C5283C
:02400E00323D41
:00000001FF
